:0200000480007A
:100000006F000005732F2034930F80006308FF03F7
:10001000930F90006304FF03930FB0006300FF038E
:10002000130F000063040F0067000F00732F2034CC
:1000300063540F006F00400093E19153171F0000BD
:1000400023223FFC171F000023200FFC6FF01FFF2F
:100050009300000013010000930100001302000050
:100060009302000013030000930300001304000038
:100070009304000013050000930500001306000020
:100080009306000013070000930700001308000008
:10009000930800001309000093090000130A0000F0
:1000A000930A0000130B0000930B0000130C0000D8
:1000B000930C0000130D0000930D0000130E0000C0
:1000C000930E0000130F0000930F0000732540F102
:1000D0006310050097020000938202017390523072
:1000E000735044749702000093820201739052305F
:1000F00073500018970200009382420273905230AE
:100100009B021000939252039382F2FF7390023B82
:100110009302F0017390023A73504030970200004E
:1001200093824201739052307350203073503030BC
:100130009301000097020000938202ED7390523009
:10014000130510001315F501635C05000F00F00F97
:10015000930110009308D005130500007300000000
:1001600093020000638A020073905210B7B200003D
:100170009B829210739022307350003097020000DF
:100180009382420173901234732540F17300203042
:1001900093012000930000001301000033A720000A
:1001A00093030000631A774A930130009300100014
:1001B0001301100033A7200093030000631E77484B
:1001C00093014000930030001301700033A720001A
:1001D000930310006312774893015000930070005E
:1001E0001301300033A72000930300006316774605
:1001F00093016000930000003781FFFF33A72000C8
:1002000093030000631A774493017000B7000080E5
:100210001301000033A7200093031000631E7742F0
:1002200093018000B70000803781FFFF33A72000D3
:100230009303100063127742930190009300000033
:10024000378100001B01F1FF33A72000930310004A
:10025000631477409301A000B70000809B80F0FFFB
:100260001301000033A72000930300006316773EBC
:100270009301B000B70000809B80F0FF3781000041
:100280001B01F1FF33A72000930300006316773CA6
:100290009301C000B7000080378100001B01F1FF0F
:1002A00033A72000930310006318773A9301D0001E
:1002B000B70000809B80F0FF3781FFFF33A720004D
:1002C00093030000631A77389301E0009300000065
:1002D0001301F0FF33A7200093030000631E77365D
:1002E0009301F0009300F0FF1301100033A72000EA
:1002F0009303100063127736930100019300F0FF1F
:100300001301F0FF33A72000930300006316773436
:10031000930110019300E0001301D000B3A020006E
:1003200093030000639A7032930120019300B000A0
:100330001301D00033A1200093031000631E71301D
:10034000930130019300D000B3A01000930300008C
:100350006394703093014001130200009300B000D9
:100360001301D00033A7200013030700130212006B
:1003700093022000E31452FE93031000631E732CBB
:1003800093015001130200009300E0001301D0001C
:1003900033A720001300000013030700130212000C
:1003A00093022000E31252FE930300006316732AA7
:1003B00093016001130200009300C0001301D000FC
:1003C00033A72000130000001300000013030700F0
:1003D0001302120093022000E31052FE9303100058
:1003E000631C732693017001130200009300E00068
:1003F0001301D00033A72000130212009302200043
:10040000E31652FE930300006318772493018001E2
:10041000130200009300B0001301D000130000008D
:1004200033A720001302120093022000E31452FEAF
:1004300093031000631277229301900113020000CE
:100440009300F0001301D00013000000130000001F
:1004500033A720001302120093022000E31252FE81
:1004600093030000631A771E9301A001130200009A
:100470009300A000130000001301D00033A7200058
:100480001302120093022000E31452FE93031000A3
:100490006314771C9301B001130200009300000164
:1004A000130000001301D0001300000033A7200048
:1004B0001302120093022000E31252FE9303000085
:1004C000631C77189301C001130200009300900091
:1004D00013000000130000001301D00033A7200018
:1004E0001302120093022000E31252FE9303100045
:1004F000631477169301D001130200001301D0009A
:100500009300100133A72000130212009302200071
:10051000E31652FE93030000631077149301E00189
:10052000130200001301D0009300800013000000AC
:1005300033A720001302120093022000E31452FE9E
:1005400093031000631A77109301F0011302000067
:100550001301D000930020011300000013000000DD
:1005600033A720001302120093022000E31252FE70
:10057000930300006312770E930100021302000040
:100580001301D000130000009300700033A7200077
:100590001302120093022000E31452FE9303100092
:1005A000631C770A93011002130200001301D000AC
:1005B00013000000930030011300000033A7200057
:1005C0001302120093022000E31252FE9303000074
:1005D0006314770893012002130200001301D00076
:1005E00013000000130000009300600033A72000F8
:1005F0001302120093022000E31252FE9303100034
:10060000631C7704930130029300F0FF3321100044
:100610009303000063127104930140029300F0FF02
:1006200033A100009303100063187102930150027C
:10063000B3200000930300006390700293016002F6
:10064000930000011301E00133A020009303000098
:1006500063147000631030020F00F00F638001001C
:100660009391110093E111009308D00513850100C7
:10067000730000000F00F00F930110009308D005E5
:100680001305000073000000731000C0000000009C
:10069000000000000000000000000000000000005A
:1006A000000000000000000000000000000000004A
:0C06B0000000000000000000000000003E
:1010000000000000000000000000000000000000E0
:1010100000000000000000000000000000000000D0
:1010200000000000000000000000000000000000C0
:1010300000000000000000000000000000000000B0
:081040000000000000000000A8
:040000058000000077
:00000001FF
